:1000000018308A00DF2E0000FF00030E8301A100DC
:100010000A08A0008A010408A2007708A300780853
:10002000A4007908A5007A08A6007B08A70083131E
:1000300083128C308400001C1F280C1832282208E0
:1000400084002308F7002408F8002508F900260892
:10005000FA002708FB0020088A00210E8300FF0E0B
:100060007F0E09008A110A1241280A108A100A110B
:10007000820700340034103430348A3400340034C1
:100080002D34061D452806114628061564000C105F
:100090008A110A121F28871087162130F700F70BE4
:1000A0004F2800348C1A5628640052288C1E56287B
:1000B0001A088316CB008312981C64281A0883162A
:1000C000CB0083121812181683164B08F8008312FF
:1000D00000342908073C031D722807300C1E6E28C7
:1000E0009900B12805308316B9003908063C031978
:1000F000B0283908053C031DAA282930BB0083120B
:100100006F088316B800043083120C1E85289900EE
:100110006F080C1E892899008316BA0183126F0894
:1001200083163A020318A4283B0884000008BC0088
:1001300083120C1E9928990083163B08840000083E
:10014000B806BB0ABA0A8E28380883120C1EA628E5
:10015000990083168312522078088316B9007528F7
:10016000831200349030A9000130AA003930AB006E
:10017000831681138312861DC0280230AC00C2286A
:100180000130AC000430EF0069200034D43084002A
:1001900000080319D8280630F800F701F70BCE281D
:1001A000F80BCD287B30F700F70BD428800BCB2839
:1001B00000349130A9000230EF0069202A08F700CE
:1001C000F7080319F828013077020319FE280230D6
:1001D0007702031904290330770203190A2906302C
:1001E00077020319102907307702031916291D29F0
:1001F000813083169900263098001F2940308316DD
:100200009900263098001F29203083169900263047
:1002100098001F29153083169900263098001F2951
:100220000A3083169900263098001F29043083165F
:100230009900263098001F29831283161F29023047
:10024000D4008312C6208A110A166528F701F80126
:100250008316510803105218F707F70CF80CD21840
:10026000F707F70CF80C5219F707F70CF80CD2192E
:10027000F707F70CF80C521AF707F70CF80CD21A1C
:10028000F707F70CF80C521BF707F70CF80CD21B0A
:10029000F707F70CF80C831200349230A9006F08AE
:1002A000413C03196C290130AA008316B1013108C1
:1002B0003F3C031C6A2902303107293E8400310883
:1002C000D1000530D20083122621780880008316E1
:1002D000B10A5729A32983128316B10131083F3C83
:1002E000031C852901303107293E84000008B30032
:1002F0003108D1000530D2008312262178088316F8
:100300003302031D8529B10A6E2931083F3C031CC5
:100310008B2901308C2900308312AA008316B10189
:1003200031083F3C031CA32902303107293E8400D9
:100330003108D1000530D2008312262178088000D0
:100340008316B10A902942308312EF0069208A1186
:100350000A166D289530A9000508AA000608AB000A
:100360000708AC00053083169F0083121F08383938
:10037000C1389F000030F8001F08C73978049F007B
:10038000A630F700F70BC22900001F151F19C62958
:100390001E08AD000830F8001F08C73978049F0018
:1003A000A630F700F70BD22900001F151F19D62918
:1003B0001E08AE000630EF00692000346F08073CCD
:1003C000031DF5292A088316850083122B0883163E
:1003D000860083122C088316870083122D0885005F
:1003E0002E0886002F088700AA218A110A16752870
:1003F0002A088316B2002B30B300B10102308312F9
:100400006F02831631020318312A3208B20AB4008F
:100410003308B30A84000008B500340883120317B8
:100420008D008F01831603133508831203178C0088
:1004300083168C130C15831203130B08F7008B1310
:100440008316031755308D00AA308D008C148C183C
:10045000272A0C117708831203138B048316B10A21
:10046000FE2907308312A9000130EF0069208A11AC
:100470000A1685282A088316B2002B30B30083128F
:100480002B08EF008316B10183126F088316310227
:1004900003185E2A3308B30A84003208B20AB50092
:1004A000831203178D008F0183168C130C14831293
:1004B0000C08800083160313B10A442AE330831228
:1004C000A9000230EF0769208A110A168D28E5304D
:1004D000A9000230AA00EF0069208A110A169528A7
:1004E000E730A9004630AA000230EF0069208A11E7
:1004F0000A169D288712003419308316AA0063302B
:10050000AB000330AC000230AD002E10AF01233041
:100510003502FE3E0318A32A023E8312A72A0130A9
:100520008316A100A201A3010530A400A501A60124
:10053000A32A8316A1016430A200A301A401A5018E
:10054000A601A32A831683128A110A12512B0A10BC
:100550008A140A1182078F2A992A83163308A00069
:100560000130A100A201A3010530A400A500A6014D
:100570000830A7000730A8004030A9002030200232
:10058000ED3E0318542B133E8312672B0130831664
:10059000AD002E10AF01542B01308316AD002E1488
:1005A000AF01542B8316AD012E10AF01542B8316CF
:1005B000AD012E14AF01542B01308316A100A2010E
:1005C000A3016430A4000530A500A6010830A700EF
:1005D0000730A8002030A9002008223C031DF52A7E
:1005E0000130AD002E14AF00F92AAD012E140130F8
:1005F000AF00542B01308316A100A201A301643087
:10060000A4000530A500A6012030A7001F30A800D7
:100610004030A9002008253C031D132B0130AD00FC
:100620002E14AF00172BAD012E140130AF00542B48
:1006300001308316A100A201A3016430A40005309B
:10064000A500A6014030A7003F30A8004030A90017
:100650002008263C031D312B0130AD002E14AF00C5
:10066000352BAD012E140130AF00542B0230831610
:10067000A100A201A3017830A4001E30A500A601AC
:100680001030A7000F30A8001030A9000130AD00D5
:100690002E140230AF00542B83163308B50083129A
:1006A0007C2A8316542B831683178316B4013408CF
:1006B0003F3C031C612BA030340784008001B40A46
:1006C000572B7410831283138A110A12AA2B0A144F
:1006D0008A140A118207CC2ACC2ADC2A4C2B4C2BF8
:1006E000FA2A182B362BC62ACC2A532BD22AD72AE1
:1006F000532BD72AD72ADC2AFA2A182B80308316C4
:10070000870581308704D93086050616DB308505DC
:100710001B30850405158516861483128711071270
:100720004B207A2287142130F700F70B952B4B20B2
:100730007A2287142130F700F70B9C2B20302802F7
:10074000FF3E0318AB2B013EAE2B83163208B300DD
:100750008312AD2AAB2B8A110A12BF2B0A148A14FA
:100760000A118207A52B2A088316B1003108E03947
:100770008312A80083163108B20083127E2B073043
:10078000A9000130EF0069208A110A16A5288316F6
:10079000311083122A080139003A0319D62B6F0849
:1007A000023C031DD62B83163114831200308316AE
:1007B00031180130B200B30083124B2007110C3006
:1007C00097000030F80004389200773083169200CA
:1007D000B3080319F32B3C30831295001708CF3967
:1007E0009700F92B83162030831295001708CF3914
:1007F00097004B2004308316B200AF30D400831230
:10080000C6208316B20BFD2B07308312A9000130DE
:10081000EF0069208A110A16AD2807119701970188
:100820004B200730A9000130EF0069208A110A1619
:10083000B5288316DF015F08033C031C2E2C031030
:10084000DE0C0318272C83120712292C831683121F
:100850000716871587118316DF0A1B2C83120034B5
:1008600087118316E30163080F3C031C472C031018
:10087000E20CE10C0318402C83120712422C831661
:1008800083120716871587118316E30A332C640039
:1008900083120034D9308316DD00DE01831219245F
:1008A000023083165D0784000008DE000E30E00091
:1008B0005E08DF006008E2005E08E1008312302479
:1008C0008316DE01831219246E308316E200F8309D
:1008D000E100831230248316DE01831219240130D3
:1008E00083165D0784000008DE000E30E0005E081D
:1008F000DF006008E2005E08E10083123024831606
:10090000DE01831219246E308316E200F730E10015
:10091000831230248316DE018312192483165D08A6
:1009200084000008DE000E30E0005E08DF00600892
:10093000E2005E08E100831230248316DE01831298
:1009400019246E308316E200F630E1008312302461
:100950000034E030840000080319B32CB12C0000EF
:100960000000800BAF2C00348316DC013C30DB0030
:10097000DA010430D90083124A240C308316DE00D9
:100980008312192483163708E2003608E100831227
:1009900030248316DE01831219248316E201E1015B
:1009A000831230248316DE01831219248316230850
:1009B0002507B800D4008312C62083162408260712
:1009C000B800E0008312A9248316E201E10183123A
:1009D000302400348316DC013C30DB00DA010530C2
:1009E000D90083124A240C308316DE0083121924A6
:1009F00083163708E2003608E1008312302483169C
:100A0000DC013C30DB00DA010430D90083124A24D7
:100A10000C308316DE008312192483163708E20097
:100A20003608E100831230248316DE018312192474
:100A30008316E201E101831230248316DE01831262
:100A40001924831623082507B800D4008312C62072
:100A5000831624082607B800E0008312A924831611
:100A6000E201E10183123024003483163408FD3E94
:100A70000318472D033E83124B2D01308316B70018
:100A80008A30B6008312EA248316472D8316831218
:100A90008A110A12FF2D0A148A100A1582073D2DA9
:100AA000462D3D2D83162F08FD3E0318022E033ED2
:100AB0008312062E83163208B4003408F700013082
:100AC0007702831203196C2DF7080319732D023076
:100AD000770203198A2D902D8316B7018130B60055
:100AE0008312B424912D8316B7018330B60083128C
:100AF000B42488308316B50035088F3C031C882D3C
:100B0000B7013508B6008312B4248316B50A7C2DCC
:100B10008312912D8316B7018030B6008312B4245E
:100B2000912D8316022E83163208B4003408F70084
:100B30000130770283120319A52DF7080319AC2D94
:100B4000023077020319F02DF72D8316B701843098
:100B5000B6008312EA24F82D8316B7018130B6005F
:100B60008312EA248316B7018230B6008312EA2486
:100B700001308316B7008030B6008312EA240230B9
:100B80008316B7008030B6008312EA24043083163F
:100B9000B7008030B6008312EA2408308316B7000D
:100BA0008030B6008312EA2410308316B7008030FC
:100BB000B6008312EA2420308316B7008030B600D6
:100BC0008312EA2440308316B7008030B6008312C7
:100BD000EA2480308316B700B6008312EA24F82D89
:100BE0000F308316B7008730B6008312EA24F82D41
:100BF0008316022E83163208B4008312352D831615
:100C0000022E831683128A110A12192E0A108A14D0
:100C10000A1582075A2D932DFA2D20302802FF3E07
:100C200003181A2E013E1F2E83163108B2008312BC
:100C3000522D1A2E871107128A110A12292E0A1014
:100C40008A140A158207142E2A088316B10083120B
:100C50000D2E0730A9000130EF0069208A110A1615
:100C6000BD288316D608031D392E55082F3C0318BE
:100C70004C2ED608031D4C2E5508303C031C4C2E20
:100C8000031D492ED408031D4C2E53080D3C031C94
:100C90004C2ED801D7014F2E1030D800D701DE01DD
:100CA000831219248E308316E200A630E1008312ED
:100CB00030248316DE0183121924EF308316E200FC
:100CC000E101831230248316DE0183121924F830E7
:100CD0008316E200E101831230248316DE018312C1
:100CE000192483165708A638D90058088C38DA001A
:100CF000E2005908E1008312302483165608DC0014
:100D00005508DB005408DA005308D90083124A243E
:100D100000348316DE018312192484308316E20026
:100D2000A630E100831230248316DE0183121924D9
:100D300088308316E200A630E10083123024831647
:100D4000DE01831219240E308316E2005530E100D3
:100D5000831230248316DE01831219246E30831629
:100D6000E200A730E100831230248316DE018312F3
:100D700019240E308316E200AA30E10083123024D9
:100D80008316DE01831219246E308316E200A73029
:100D9000E100831230248316DE018312192482308D
:100DA0008316E200A630E100831230248316DE01B0
:100DB000831219248316E201E10183123024831681
:100DC000DE0183121924831623082507D300D400DB
:100DD0008312C620831624082607D300E00083125E
:100DE000A9248316E201E101831230248316DE0177
:100DF0008312192494308316E200A630E100831296
:100E0000302400348316CD08031D0A2F4C081F3CE4
:100E10000318342FCD08031D332F4C082F3C031C1F
:100E2000332F7418332FDC013C30DB00DA0106303D
:100E3000D90083124A240C308316DE008312192451
:100E40008316E201E1018312302483164D08D60097
:100E50004C08D5004B08D4004A08D3008312312631
:100E6000892674148316B92F0030CA05F030CB05DB
:100E70001F30CC050030CD05FA014D0CF9004C0CAB
:100E8000F8004B0CF700F90CF80CF70CF90CF80C07
:100E9000F70CF90CF80CF70C7708CE004E0CCF00CD
:100EA000CF0CCF0C1F30CF054E080739F8000130AA
:100EB000CE00F8080319602F0310CE0DF80B5C2F3D
:100EC0008317A03083164F07840000084E05003AB0
:100ED000031DB72FA0304F07840000084E04800088
:100EE000831283138316D101D001D108031DB72FBC
:100EF00050083F3C031CB72F6400D20152083F3C0E
:100F0000031CB32F6400DC013C30DB00DA01063047
:100F1000D90083124A240C308316DE008312192470
:100F20008316E201E1018312302483164D08D600B6
:100F30004C08D5004B08D4004A08D3008312312650
:100F4000892683162908CA07003003180130CB0709
:100F5000003003180130CC07003003180130CD07F2
:100F60002908D2077E2FD00A0319D10A752F8313BF
:100F70008316831200348316D1015108023C031CEE
:100F8000D02F0310D00C0318C92F83120712CB2FB8
:100F9000831683120716871587118316D10ABD2F72
:100FA0000310D00C0318D82F83120712DA2F8316E0
:100FB00083120716871583162108D4008312C620D2
:100FC00083162208E0008312A924871183162308C0
:100FD000D4008312C62083162408E0008312A924BB
:100FE000003400308C1A0130F800003429080C1E3F
:100FF000F72F99002908EE060034FF3FFF3FFF3F1F
:1010000083160716D10151080F3C031C15288312C3
:1010100087158711071A0E2803100F28031483164B
:1010200050088400800CD10A03280712831287110C
:10103000003483164C08013C03187728CD01023098
:101040004C024D02031841280D30DE008A11831234
:1010500019248A1583164B08CB0ACB0A8400840A0C
:101060000008CF0084030008CE004F08E2004E08BD
:10107000E1008A11831230248A1502308316CD07CD
:101080001F280F30DE008A11831219248A15831657
:101090004B08CB0ACB0A8400840A0008CF008403E3
:1010A0000008CE004F08E2004E08E1008A118312CA
:1010B00030248A158316D0018A118312BB278A1522
:1010C0008316E201E1018A11831230248A150D3062
:1010D0008316DE008A11831219248A15FF308316C5
:1010E000E200E1008A11831230248A1583168312EC
:1010F000003420302802FF3E0318132B013E182B2A
:1011000083163908BF003808BE003708BD0036080E
:10111000BC003A08C0003B08C100AD08031DD4283C
:101120003F08CD003E08CC003D08CB003C08CA007B
:101130008A11831202278A15831641083C07C200D0
:101140003D08C300003003180130C3073E08C40047
:10115000003003180130C4073F08C50000300318F1
:101160000130C50701304202C6004308C700003005
:10117000031C0130C7024408C8000030031C0130C2
:10118000C8024508C9000030031C0130C9024908E3
:10119000CD004808CC004708CB004608CA008A1199
:1011A000831202278A158316DC013C30DB00DA014A
:1011B0000630D9008A1183124A248A150C3083160E
:1011C000DE008A11831219248A158316E201E101D7
:1011D0008A11831230248A1583163F08D6003E08F0
:1011E000D5003D08D4003C08D3008A118312312673
:1011F0008A158316BF08031D01293E082F3C0318DA
:101200000C2ABF08031D0C2A3E08303C031C0C2A84
:10121000031D1129BD08031D0C2A3C080D3C031CAD
:101220000C2A2D08F700F708831203192029013032
:1012300077020319202902307702031978290A2A34
:1012400083164008C2004108C3004208C500C4011B
:1012500043084402031876290F30DE008A118312F6
:1012600019248A15831645088400840A0008C700DB
:1012700084030008C6004708E2004608E1008A111E
:10128000831230248A158316D0018A118312BB275A
:101290008A158316E201E1018A11831230248A152E
:1012A0008316D0018A118312BB278A152A30831630
:1012B000E200F630E1008A11831230248A15831689
:1012C000DE018A11831219248A158316E201E101D5
:1012D0008A11831230248A15831644080139F700D5
:1012E0000310F70D7708C507C40A28290B2A0B2A13
:1012F00083164008C2004108C3004208C40003101E
:10130000C30CC3080319082A4408C40AC40A840089
:10131000840A0008FA0084030008C5007A08C600A1
:101320002B08C8000D30DE008A11831219248A159B
:1013300083164608E2004508E1008A118312302432
:101340008A158316D0018A118312BB278A1583164A
:10135000E201E1018A11831230248A150C308316D0
:10136000DE008A11831219248A1583164608E200CA
:101370004508E1008A11831230248A158316D001B2
:101380008A118312BB278A158316E201E1018A11B3
:10139000831230248A158316C80BCF29D1298312D2
:1013A000AE290E30DE008A11831219248A158316A5
:1013B0004608E2004508E1008A11831230248A15AC
:1013C0008316D0018A118312BB278A158316E20186
:1013D000E1018A11831230248A1509308316DE0058
:1013E0008A11831219248A15C7308316D0008312FC
:1013F000002009308316DE008A11831219248A1511
:10140000C7308316D000831200208316C3038129BE
:101410000B2A83128316112B2D08F700F70883126D
:1014200003191B2A0130770203191B2A02307702A5
:101430000319612A102B83163F08C5003E08C4001B
:101440003D08C3003C08C2004008C6004108C70070
:1014500042082805C900C9080319412A490827027A
:10146000CA0047020318362A4708CA004608CB00BC
:101470004A08CC008312192083164A08C7024A087A
:10148000C60747082805C8002808FF3AC705C70847
:101490000319562A4608CB002708CC0083121920CE
:1014A00083162708C6072708C702472AC808031952
:1014B000602A4608CB004808CC0083121920831606
:1014C000112B83163F08C5003E08C4003D08C30029
:1014D0003C08C2004008C6004108C7004608C800D2
:1014E0000310C70CC70803190E2B4808C80AC80AFE
:1014F0008400840A0008FA0084030008C9007A08FE
:10150000CA002A08CF000D30DE008A118312192488
:101510008A1583164A08E2004908E1008A118312FD
:1015200030248A158316D0018A118312BB278A15AD
:101530008316E201E1018A11831230248A150A30F0
:101540008316DE008A11831219248A15CD30831682
:10155000D0008312002008308316DE008A11831227
:1015600019248A15CE308316D000831200208316EA
:101570004D08CC004E08CB00CF030319C72A4908F9
:101580004B02031D832A4A084C02031D832A4F087D
:101590002A02D0002C08D1005008D2008A118312F0
:1015A00026218A1578088316CF000C30DE008A11B8
:1015B000831219248A1583164A08E2004908E100BB
:1015C0008A11831230248A158316D0018A1183125E
:1015D000BB278A158316E201E1018A1183123024A8
:1015E0008A158316CF0BD52A0930DE008A118312A3
:1015F00019248A15CD308316D000831200200930BB
:101600008316DE008A11831219248A15CD308316C1
:10161000D000831200208316C703722A112B831275
:1016200083168312132B871107128A150A123E2B79
:101630000A148A140A11820780288316B4018312BF
:101640002C088316B30083122B088316B200831272
:101650002A088316B100043083126F028316B50086
:101660003408B9003308B8003208B7003108B600B2
:101670002D30BA003508BB00831279280730A90045
:101680000130EF008A1169208A158A110A16C628CE
:1016900020302802FF3E0318802B013E852B831645
:1016A0003808BE003708BD003608BC003508BB004E
:1016B0003908BF003A08C0003E08D6003D08D500F2
:1016C0003C08D4003B08D3008A11831231268A15C6
:1016D0008316C1014008410203187E2B0930DE0049
:1016E0008A11831219248A1583163F084107C20004
:1016F000D000831200208316C10A6A2B8312802B2C
:10170000871107128A150A12AC2B0A148A140A11BF
:1017100082074F2B8316B40183122C088316B30063
:1017200083122B088316B20083122A088316B10095
:1017300083122D08EF0083163408B8003308B70071
:101740003208B6003108B5002D30B90083126F0899
:101750008316BA008312482BC430A9000430EF0767
:101760008A1169208A158A110A16D0288316DE018B
:101770008A11831219248A1583164308C4000E3077
:10178000C500E2004308E1008A11831230248A1563
:101790008316DE018A11831219248A156E3083168E
:1017A000E200A830E1008A11831230248A158316E2
:1017B000DE018A11831219248A1584308316E2000F
:1017C000A630E1008A11831230248A158316DE01C7
:1017D0008A11831219248A150E308316E2005530BF
:1017E000E1008A11831230248A158316DE018A11E2
:1017F000831219248A156E308316E200A730E100A7
:101800008A11831230248A158316DE018A1183120D
:1018100019248A150E308316E200AA30E1008A11DD
:10182000831230248A158316DE018A11831219244B
:101830008A156E308316E200A730E1008A11831208
:1018400030248A158316DE018A11831219248A1521
:1018500082308316E200A630E1008A118312302420
:101860008A15003420302802FF3E0318F12D013E76
:10187000F62D83163508B9003408B8003608BA00CA
:101880003708BB0000302E180130F700F70883122C
:1018900003194F2C013077020319F22CEE2D831619
:1018A0003908BD003808BC003A08BE003B08BF003C
:1018B000DE018A11831219248A159E308316E200F4
:1018C000A630E1008A11831230248A158316DE01C6
:1018D0008A11831219248A159C308316E200A630DF
:1018E000E1008A11831230248A158316C0013F0853
:1018F00040020318F12CDE018A11831219248A1583
:1019000083163D08FA003C08BC0A0319BD0AC10051
:101910007A08C2004108F70042080039FA0041087D
:10192000C3007A080E38C400E2004108E1008A11C1
:10193000831230248A158316DE018A11831219243A
:101940008A156E308316E200A930E1008A118312F5
:1019500030248A1583163E08400784000008C10021
:10196000C3008312B6238316DE018A118312192461
:101970008A158316E201E1018A11831230248A1547
:101980008316DE018A11831219248A15831623080F
:101990002507C100D4008A118312C6208A15831638
:1019A00024082607C100E0008A118312A9248A15A1
:1019B0008316E201E1018A11831230248A1583160D
:1019C000DE018A11831219248A1594308316E200ED
:1019D000A630E1008A11831230248A158316C00ACA
:1019E000772CEF2D83163908BD003808BC003A0863
:1019F000BE003B08BF00DE018A11831219248A153C
:101A00009E308316E200A630E1008A118312302452
:101A10008A158316DE018A11831219248A159C30D7
:101A20008316E200A630E1008A11831230248A1561
:101A30008316C0013F0840020318EC2D0230C1009C
:101A4000DE018A11831219248A1583163C08F700D7
:101A50003D080039FA003C08C2007A080E38C3007D
:101A6000E2003C08E1008A11831230248A158316B3
:101A7000DE018A11831219248A156E308316E20062
:101A8000A930E1008A11831230248A158316DE0101
:101A90008A11831219248A1583163D08C200C301D6
:101AA0003D08F70043080039FA003D08C4007A08F1
:101AB0000E38C500E2003D08E1008A11831230248F
:101AC0008A158316BC0A0319BD0ADE018A11831226
:101AD00019248A156E308316E200AA30E1008A11BB
:101AE000831230248A155330F700F70B752D8316B7
:101AF0003E08400784000008C200C3008312B623DA
:101B0000831641080239003A0319C82DDE018A11F3
:101B1000831219248A1550308316E200A630E100A2
:101B20008A11831230248A151030F700F70B962D96
:101B300000008316DE018A11831219248A156E3083
:101B40008316E200F530E1008A11831230248A15F1
:101B50008316DE018A11831219248A158316E20185
:101B6000E1018A11831230248A1502308316DE00C7
:101B70008A11831219248A15C1308316D00083126A
:101B800000201030F700F70BC32D0000802D8316C6
:101B90002308D4008A118312C6208A1583162408CC
:101BA000E0008A118312A9248A158316DE018A11A6
:101BB000831219248A1594308316E200A630E100BE
:101BC0008A11831230248A151030F700F70BE62DA6
:101BD00000008316C00A1A2DEF2D8312831683127C
:101BE000F12D871107128A150A12112E0A148A1074
:101BF0000A158207392C2B088316B20083122A0893
:101C00008316B100033083126F028316B3003208CB
:101C1000B5003108B4002C30B6003308B700831289
:101C2000322C0730A9000130EF008A1169208A1593
:101C30008A110A16DA288316DE018A118312192402
:101C40008A1580308316E200A630E1008A118312E3
:101C500030248A158316DE018A11831219248A150D
:101C600050308316E200A830E1008A11831230243C
:101C70008A158316DE018A11831219248A156E30A3
:101C80008316E200F530E1008A11831230248A15B0
:101C90008316DE018A11831219248A158316E20144
:101CA000E1018A11831230248A1502308316DE0086
:101CB0008A11831219248A1583164108D0008312D1
:101CC0000020003420302802FF3E0318732F013E0D
:101CD000782F83163408B8003308B7003508B900E8
:101CE0003608BA0000302E180130F700F7088312CA
:101CF00003197F2E013077020319E52E702F83160A
:101D00003808BC003708BB003908BD003A08BE00DF
:101D1000DE018A11831219248A159E308316E2008F
:101D2000A630E1008A11831230248A158316DE0161
:101D30008A11831219248A159C308316E200A6307A
:101D4000E1008A11831230248A158316BF013E08F0
:101D50003F020318E42EDE018A11831219248A152A
:101D600083163C08FA003B08BB0A0319BC0AC000F2
:101D70007A08C1004008F70041080039FA0040081D
:101D8000C2007A080E38C300E2004008E1008A1160
:101D9000831230248A158316DE018A1183121924D6
:101DA0008A156E308316E200A930E1008A11831291
:101DB00030248A1583163D08BD0AC000C100831275
:101DC0001B268316BF0AA72E712F83163808BC0066
:101DD0003708BB003908BD003A08BE00DE018A1191
:101DE000831219248A159E308316E200A630E10082
:101DF0008A11831230248A158316DE018A11831218
:101E000019248A159C308316E200A630E1008A115D
:101E1000831230248A158316BF013E083F0203183F
:101E20006E2FDE018A11831219248A1583163B084E
:101E3000F7003C080039FA003B08C0007A080E3869
:101E4000C100E2003B08E1008A11831230248A15A8
:101E50008316DE018A11831219248A156E308316C7
:101E6000E200A930E1008A11831230248A1583161A
:101E7000DE018A11831219248A1583163C08C000DA
:101E8000C1013C08F70041080039FA003C08C200D3
:101E90007A080E38C300E2003C08E1008A11831280
:101EA00030248A158316BB0A0319BC0ADE018A1185
:101EB000831219248A156E308316E200AA30E100DD
:101EC0008A11831230248A1583163D08BD0AC0008A
:101ED000C10083121B268316BF0A0D2F712F831298
:101EE00083168312732F871107128A150A12942FF3
:101EF0000A148A140A158207692E2B088316B20069
:101F000083122A088316B10083122C08EF0083166F
:101F10003208B4003108B3002C30B50083126F08CA
:101F20008316B6008312622EE230A9000330EF0759
:101F30008A1169208A158A110A16E4288A114B2011
:101F40008A15D030A900AA01AB01AC01AD01053062
:101F5000EF008A1169208A158A110A16EE288A1163
:101F60007A228A15D030A9000130AA00AB01AC0159
:101F7000AD010530EF008A1169208A158A110A1611
:101F8000F82883165F1464008312071EDA2F64009A
:101F900083165E08DE03003A031DD32F5F10831201
:101FA000DA2FD92F8316FF30E0008A118312A9247B
:101FB0008A15C52F003083165F180130F800831290
:101FC000003408300C1EE22F990083164808831253
:101FD0000C1EE82F9900003403300C1EED2F9900E1
:101FE0008316380883120C1EF32F990083163808C5
:101FF0008312EE000034EE060034FF3FFF3FFF3F48
:1020000001308316B000B4012930B500B408031DB7
:1020100056280A12831252200A1678088316B10035
:102020003108043C03191C280A12831252200A1694
:1020300078088316B10010280A12831252200A165B
:102040007808EF008316B300B20183126F0883167D
:10205000320203183D283508B6000A1283125220B6
:102060000A16831636088400780880003508840034
:102070000008B306B50AB20A25280A1283125220B4
:102080000A1678088316B306031D4F280130B400E2
:10209000063083120C1E4A289900542883160530F6
:1020A00083120C1E512899008316062883122908D2
:1020B000103C031D5F280A12B2200A16FE282908C8
:1020C000113C031D67280A12D9280A16FE28290880
:1020D000123C031D6F280A124D290A16FE282908F2
:1020E000143C031D77280A12DE290A16FE28290847
:1020F000153C031D7F280A12AA210A16FE2829086A
:10210000173C031D87280A12F8290A16FE282908F9
:10211000183C031D8F280A123A2A0A16FE2829089D
:102120001A3C031D97280A12672A0A16FE28290856
:102130001B3C031D9F280A12702A0A16FE28290834
:10214000413C031DA7280A12B32B0A16FE282908B2
:10215000403C031DAF280A12C72B0A16FE28290887
:10216000473C031DB7280A120D2C0A16FE28290821
:10217000433C031DBF280A12242E0A16FE282908F4
:10218000423C031DC9280A128A151D2B0A168A1102
:10219000FE282908443C031DD3280A128A158A2BDD
:1021A0000A168A11FE282908453C031DDD280A125B
:1021B0008A15FB2D0A168A11FE282908463C031DA4
:1021C000E7280A128A157D2F0A168A11FE28290887
:1021D000503C031DF1280A128A159E2F0A168A11F7
:1021E000FE282908513C031DFB280A128A15AF2F2F
:1021F0000A168A11FE288316B0018312831630084E
:10220000F80083128A150A16482F8316560DD70038
:10221000D70DD70DF830D7050716FF30DE000A12AC
:102220008A158312C1270A168A118316D901D8018B
:1022300059087102031C2A29031D2229580870021B
:10224000031C2A290230F700F70B2429D80A0319A6
:10225000D90A1829831287158316D901D80159087C
:102260007102031C4229031D392958087002031CFE
:1022700042290630F700F70B3B290000D80A031962
:10228000D90A2F298312071A472903104829031452
:102290008316DA0DDB0DDC0D07128312071283168D
:1022A000560B58290310D20D031C582907166D2907
:1022B0005608023C031D63290310D20DD30D031CE5
:1022C000632907166D295608033C031D6D29031069
:1022D000D20DD30DD40D0318071683128711831660
:1022E000D901D80159087102031C8529031D7C29D5
:1022F00058087002031C85290630F700F70B7E2969
:102300000000D80A0319D90A72290716D70B2A29FF
:1023100007165A08F7005B08F8005C08F9005D082A
:10232000FA00831200348316BB01BC010230F100B5
:102330007130F000FF30DE000A128A158312C127C7
:102340000A168A11F8080319072A8316D501D40141
:102350001030D300D2010230D6008312052183163B
:1023600007168312071AB2298316BC01BB01831218
:102370008715F3010130F200071AC729F20A031981
:10238000F30A720873040319C7296400BC29071AE9
:10239000D229F20A0319F30A720873040319D22925
:1023A0006400C7298312071EE4298316BB0A031998
:1023B000BC0A3B083C040319E42912306400FF3EC8
:1023C000031DDE290000D2298312871172087304CD
:1023D0000319012A83163B083C04031DF1298312CB
:1023E000012A3C0CF1003B0CF000F10CF00CF10C5C
:1023F000F00CF10CF00CF10CF00C0730F105062A92
:1024000083120230F1007130F000831683128316BC
:102410003B08F8003C08F9008312003483160511CC
:10242000831205158316851283128516831686106E
:10243000831286140230F1007130F000203028023F
:10244000FF3E0318612A013E822A0A124B200A1617
:1024500087150A127A220A161030F700F70B2E2A77
:1024600000008711FF308316DE000A128A158312DE
:10247000C1270A168A110A124B200A1687150A125A
:102480007A220A161030F700F70B442A0000871151
:102490008316D501A030D400D301D2010330D60079
:1024A000831205211F30F9050030FA057A088316DA
:1024B000BA007908B9007808B8007708B700831225
:1024C000612A9321FF308316DE000A128A158312D7
:1024D000C1270A168A11F808031D752A8316BA0146
:1024E000FF30B900B800B700831283163708F70031
:1024F0003808F8003908F9003A08FA0083128A11FE
:102500000A168C2A0A108A140A118207252AB23068
:102510008316B60083120E2A7A088316B50079084E
:10252000B4007808B3007708B200D0308312A90055
:102530008316DE010A128A158312C1270A168A1130
:10254000F8080319A52A0030A62A0130AA0083162C
:102550003608B60A840000088312AB0083163608DA
:10256000B60A840000088312AC0083163608840083
:1025700000088312AD000530EF000A1269200A1628
:102580008A150A16792E8316BA01FF30B900B800F1
:10259000B700DE010A128A158312C1270A168A11B2
:1025A000F808031D032B8715A630F700F70BD62A72
:1025B0000000871120302802FF3E0318FA2A013E4E
:1025C000102B8316D501A030D400D301D2010330E3
:1025D000D600831205211F30F9050030FA057A086C
:1025E0008316BA007908B9007808B8007708B700F0
:1025F0008312FA2AFF308316DE000A128A1583122C
:10260000C1270A168A1183163708F7003808F80020
:102610003908F9003A08FA0083128A110A161A2BAF
:102620000A148A140A118207E12AB2308316B6000E
:102630008312C32A7A088316B5007908B400780893
:10264000B3007708B200D0308312A9008316DE01F0
:102650000A128A158312C1270A168A11F80803196B
:10266000332B0030342B0130AA0083163608B60A0B
:10267000840000088312AB0083163608B60A840073
:1026800000088312AC008316360884000008831209
:10269000AD000530EF000A1269200A168A150A16E5
:1026A000812E0408F8000830F7000718552B831610
:1026B000CC01F7176D2BF7136D2B0310831207183E
:1026C00003148316CC0C77176D2B7713F70B5D2B48
:1026D000780884004C08F800842B02308400003015
:1026E000F71B5530F800F80B732B840B6F2BAB30B6
:1026F000F71B2E30F800F80B7B2B00000000F71BB7
:102700005B2B771B652B5D2B83128A150A16A62877
:1027100007100830F800000000000000F817A12B97
:10272000F8138316C90C831203180714031C07102F
:102730007817A12B7813F80B912B000000000000F4
:1027400007140230F7008401840BA42BF70BA32B92
:10275000AD308400840BAA2B00000000F81B902BE6
:10276000781B9A2B8A150A164229FF308316C60059
:10277000C700C800C901DE010A128A158312C127E9
:102780000A168A11F8080319E52B20302802FF3EAB
:102790000318E52B013EF02B8316D501A030D400A1
:1027A000D301D2010330D600831205211F30F90571
:1027B0000030FA057A088316C9007908C80078083D
:1027C000C7007708C6008312E52B83164608F7007A
:1027D0004708F8004808F9004908FA008312003455
:1027E0000A148A140A118207CC2B83163714B230CC
:1027F000B60083126F08053C031D0A2C2D08013911
:10280000003A031D072C83163710092C83128316F8
:10281000371483128316BB0183122C088316BA0067
:1028200083122B088316B90083122A088316B80076
:10283000003037180130BC003B08C0003A08BF0028
:102840003908BE003808BD003C08C1008A15831253
:1028500000288A117A088316B5007908B400780830
:10286000B3007708B200D0308312A9008316DE01CE
:102870000A128A158312C1270A168A11F808031949
:10288000432C0030442C0130AA0083163608B60AC7
:10289000840000088312AB0083163608B60A840051
:1028A00000088312AC0083163608840000088312E7
:1028B000AD000530EF000A1269200A168A150A16C3
:1028C000892EFF308316DE000A128A158312C12773
:1028D0000A168A11F80803199C2C20302802FF3EA2
:1028E00003189C2C013EBC2C8316D501C030D400AB
:1028F000D301D2010330D60083120521A630F700A0
:10290000F70B802C00008316D501A030D400D30132
:10291000D2010330D600831205211F30F9050030A3
:10292000FA057A088316BA007908B9007808B80061
:102930007708B70083129C2CFF308316DE000A1242
:102940008A158312C1270A168A11F808031DAF2CB5
:102950008316BA01FF30B900B800B700831283169E
:102960003708F7003808F8003908F9003A08FA0083
:1029700083128A110A16C62C0A108A100A158207B9
:10298000742CB2308316B6008312612C7A08831639
:10299000B5007908B4007808B3007708B200D030E9
:1029A0008312A9008316DE010A128A158312C12739
:1029B0000A168A11F8080319DF2C0030E02C0130C8
:1029C000AA0083163608B60A840000088312AB00FA
:1029D00083163608B60A840000088312AC008316FA
:1029E0003608840000088312AD000530EF000A129B
:1029F00069200A168A150A16912E031DF82C003438
:102A000084011F308305073083169F0040309900F2
:102A100026309800903083129800A001A101103058
:102A2000A2003030A3008A30A400A501A6012D30F9
:102A3000A70040308316990026309800903083120A
:102A40009800403083169900263098009030831209
:102A500098004030831699002630980090308312F9
:102A600098000F30F70007308101813084000008A2
:102A7000F0390738800064000008F03977048000DE
:102A800099256400DF26412D63008C1A492D6400CE
:102A9000452D8C1E492D1A088316A0008312981C00
:102AA000572D1A088316A0008312181218168316C1
:102AB0002008F800831200342808073C031D652D08
:102AC00007300C1E612D9900982D0530FC007C0804
:102AD000063C0319982D7C08053C031D942D2830D5
:102AE000FE006E08F60004300C1E742D99006E086E
:102AF0000C1E782D9900FD016E087D020318902DA3
:102B00007E08840000088316A00083120C1E862D08
:102B100099007E0884000008F606FE0AFD0A7C2D56
:102B200076080C1E912D990045257808FC00672D2C
:102B30000034B130A8000130EE005C250034F20111
:102B40002830F300F208031DDA2D45257808EF0040
:102B50006F08043C0319B02D45257808EF00A82D17
:102B600045257808EE006E08F100F0016E0870024D
:102B70000318C82D7308F4004525740884007808EC
:102B80008000730884000008F106F30AF00AB62DED
:102B900045257808F106F108031DD52D0130F20016
:102BA00006300C1ED12D9900D92D05300C1ED62DC6
:102BB0009900A22D00347C0803178D007D088F003A
:102BC00083168C170C140000000083120E08FA0004
:102BD0000C08F8000E08F900031300347D08143CBB
:102BE0000318F62D7D08163C03181F2E7C080317CA
:102BF0008D007D088F0083160313200883120317AE
:102C00008C00831603132108831203178E0083168A
:102C10008C170C15831203130B08F8008B13831603
:102C2000031755308D00AA308D008C140000000071
:102C30008C18182E0C117808831203138B0400349F
:102C40001F30AA052A08F0002908EF006F08033991
:102C5000F400FC30EF05F301740873020318492EE9
:102C60007008FD006F08FC00DB257908F200780889
:102C7000F1007008FD006F08FC0072088316A100C7
:102C80007108A0008312EE25EF0A0319F00AF30A77
:102C90002C2E2B30F5000330F3006E08730203185E
:102CA000812E750884000008F100840A0008F200F3
:102CB000F50AF50AF008031D702E6F08033C031C8B
:102CC000702E03106F0DF900700DFA007908203E88
:102CD0008400840A720880008403710880007B2EBF
:102CE0007008FD006F08FC0072088316A1007108CF
:102CF000A0008312EE25EF0A0319F00A0230F30751
:102D00004D2E6F080339F400F4080319AB2EF008B8
:102D1000031D8E2E6F08033C0318AB2E7408043C71
:102D20000319AB2E7008FD006F08FC00DB25790845
:102D3000F2007808F1007008FD006F08FC007208CE
:102D40008316A1007108A0008312EE25F40AEF0A91
:102D50000319F00A8E2E0730A8000130EE005C2522
:102D60000034EF016F08033C031CCD2E03106F0DE0
:102D7000F700203E8400840A0008F3008403000862
:102D8000F200FD016F08FC0073088316A1007208B1
:102D9000A0008312EE25EF0AB22ECD2E0034E430CF
:102DA000A8002030A9000230EE005C25003428087D
:102DB000A900FF30A8000230EE005C2500349F25FA
:102DC0002808313C031DE62E9925F92E2808323CAF
:102DD000031DEC2E2026F92E2808333C031DF22E6D
:102DE000B126F92E2808193C031DF82ECF26F92EFE
:102DF000D7260034FF3FFF3FFF3FFF3FFF3FFF3F2E
:102E0000B2308316B6008312B5237A088316B50054
:102E10007908B4007808B3007708B200D030831284
:102E2000A9008316DE010A128A158312C1270A1629
:102E30008A11F80803191E2F00301F2F0130AA0035
:102E400083163608B60A840000088312AB00831686
:102E50003608B60A840000088312AC0083163608D0
:102E6000840000088312AD000530EF000A126920CB
:102E70000A168A150A16992E8316C201FF30DE0043
:102E80000A128A158312C1270A168A11F808031933
:102E9000562F8316D501D401D301D2010130D600BB
:102EA0008312052177088316C20083128316420815
:102EB000F80083120034FF308316DE000A128A15F0
:102EC0008312C1270A168A11F8080319852F831661
:102ED0003F08F70040080F39FA003F08C2007A089F
:102EE0004038C300C401C5014508D5004408D400DA
:102EF0004308D3003F08D2000230D60083120521D8
:102F00003C2778088316C1008312FF308316DE0049
:102F10000A128A158312C1270A168A11F808031D9E
:102F2000952FFF308316C100831283164108F800E5
:102F3000831200346E080C1E9B2F99000A12522037
:102F40000A167808063C031D9E2F0034FF308316B6
:102F5000DE000A128A158312C1270A168A11F808A0
:102F60000319E72F83164108F70042080F39FA00CA
:102F70004108C4007A085038C500C601C701470897
:102F8000D5004608D4004508D3004408D2000230DA
:102F9000D60083120521FF308316DE000A128A153F
:102FA0008312C1270A168A1183164308C4006030B1
:102FB000C500C601C7014708D5004608D40045082A
:102FC000D3004408D2000230D60083120521003419
:102FD0002908AA00FF30A9000230EF000A12692078
:102FE0000A168A150A16D92EEF000A1269200A1647
:102FF0008A150A169C2DFF3FFF3FFF3FFF3FFF3F13
:10300000FF308316C200C300C400C501DE010A12EE
:103010008312C1270A16F8080319772820302802DE
:10302000FF3E03187728013E822983164008C90015
:103030003F08C8003E08C7003D08C600FF30CA0070
:10304000CB00CC00CD014608F7004708F80048083F
:103050001F39F90049080039FA004608CE00470830
:10306000CF0079088038D0007A08D100D500500808
:10307000D4004708D3004608D2000330D6008A1196
:10308000831205218A158316DE010A128312C127D5
:103090000A16F808031964288316D501A030D40055
:1030A000D301D2010330D6008A11831205218A157B
:1030B00077088316CA007808CB0079081F39CC003E
:1030C0007A080039CD00831283164A08F7004B08AE
:1030D000F8004C08F9004D08FA007A08C500790894
:1030E000C4007808C3007708C200831277288316CB
:1030F000C10803195629461046185629DE010A123E
:103100008312C1270A16F80803198828831656293E
:10311000C7308316C8004914C9108610831286145C
:1031200083160714F41C9928480884000130800095
:10313000D428C918D428640083120718AF2883162E
:1031400048088400CB008A118312512B8A158316FC
:103150004B08840078088000C914D32883120A120F
:103160008A11F1270A168A15F8080319C5280A12C8
:103170008A1152200A168A157808023C031DC428B9
:103180008316C91449108312D2288316DE010A124D
:103190008312C1270A16F8080319D2288316C91406
:1031A0004910831283169928003049180130F8001D
:1031B000F808031952294708F700013077028312F3
:1031C0000319E328492901308316C8000A12831223
:1031D000E1270A16C7308316C8004914C910C91858
:1031E0003129DE010A128312C1270A16F8080319D1
:1031F000FB28831631290A128A11F1270A168A152B
:10320000F80803192F2983164808CA000A128A11E0
:10321000831252200A168A1583164A0884007808F9
:103220008000480884000008083C031D262948083F
:10323000CA000A128A11831252200A168A158316AE
:103240004A08840078088000C9142E2948088400A0
:103250000008023C031D2E29C9144910831283164D
:10326000EF28003049180130F800F8080319452903
:10327000F4104708C800861407104808C9008A11CE
:103280008312882B8A1548298316F4144614831256
:10329000502983164708C8000A128312E1270A162C
:1032A000542983164614831283167C28420F5F2903
:1032B000430F5F29440F5F29C50803196929420F8D
:1032C0007629430F7629C408031D7629C508031DF6
:1032D00076298A118312B5238A157A088316C500C8
:1032E0007908C4007808C3007708C2004208F700D4
:1032F0004308F8004408F9004508FA0083128A11CF
:103300000A16292C0A148A100A1182071528293056
:103310008316B40083122B088316B30083122A0885
:103320008316B20083122C088316B60003303607CA
:10333000B700B8000A128312EC270A168316340865
:103340008400E03080000A128A118312F6270A16E0
:103350008A1583163408840083122A0880000A1212
:103360008A11F6270A168A158316340884008312F8
:103370002B0880000A128A11F6270A168A1583166E
:103380003408B7003308C0003208BF008A11831226
:103390005B278A15831637088400780880000A1294
:1033A0008A118312F6270A168A1501308316B50092
:1033B000360835020318F0293408B7008A11831241
:1033C0003C278A15831637088400780880000A1283
:1033D0008A118312F6270A168A158316B50AD82988
:1033E0008A1183129A278A158A150A16A02E2B088D
:1033F0008316B40083122A088316B3000330B20088
:1034000083126F08831632020318212A3408FA0047
:103410003308B30A0319B40AB5007A08B600293094
:10342000320784000008B7003608C2003508C10022
:103430003708C3008A118312A6278A158316B20A99
:10344000002A07308312A9000130EF000A128A1106
:1034500069200A168A158A150A16A62E83164008B0
:10346000F70041080339FA004008C2007A08203802
:10347000C300C401C5014508D5004408D400430871
:10348000D3004008D2000230D6008A1183120521F1
:103490008A158316D501D401D3010230D200013040
:1034A000D6008A11831205218A157708F8000034A6
:1034B0008316BC01FF30DE000A128312C1270A16F0
:1034C000F8080319762A20302802FF3E0318762ACE
:1034D000013E7D2A83163B08C1003A08C0008312D2
:1034E0002E2278088316BC008312762A83163C08A5
:1034F000F80083128A150A16D02A0A108A140A11B3
:1035000082076A2A29308316B40083122B08831697
:10351000B30083122A088316B20083122C08831684
:10352000B60003303607B700B8000A128312EC2742
:103530000A16831634088400E23080000A128A11C9
:103540008312F6270A168A1583163408840083121C
:103550002A0880000A128A11F6270A168A1583168D
:103560003408840083122B0880000A128A11F6277F
:103570000A168A158316B501360835020318DE2AA5
:103580003408B7003308FA003208B20A0319B30A44
:10359000B8007A08B900BB003808BA008312582A6C
:1035A000831637088400780880000A128A11831273
:1035B000F6270A168A158316B50ABC2A8A118312C1
:1035C0009A278A158A150A16AC2EFF308316DE005C
:1035D0000A128312C1270A16F80803193B2B203060
:1035E0002802FF3E03183B2B013E3E2B8316360874
:1035F000BA003508B9003708BB003808BC00BD0167
:103600003C083D020318392B3D083907BE003A0833
:10361000BF000318BF0A3F08C1003E08C000831264
:103620002E2283163B083D0784000008BE00BF0021
:10363000FF30DE000A128312C1270A16F8080319A8
:10364000362B83163F08C0003030C100C201C301D1
:103650004308D5004208D4004108D3003F08D200F7
:103660000230D6008A11831205218A158316BD0AFD
:10367000002B83123B2B8A150A16592B0A148A1425
:103680000A118207F62A2B088316B30083122A0830
:103690008316B200033083126F028316B40033081E
:1036A000B6003208B5002C30B7003408B8008312D9
:1036B000E52A0730A9000130EF000A128A116920BB
:1036C0000A168A158A150A16B22EFF308316DE00F6
:1036D0000A128312C1270A16F8080319D52B2030C5
:1036E0002802FF3E0318D52B013ED82B83163A083B
:1036F000C0003908BF003808BE003708BD003B08CD
:10370000C1003C08C2000310BF0CBE0CBD0C3D083C
:10371000F7003E08F8003F081F39F900400800395B
:10372000FA003D08C4003E08C5007908D038C6003C
:103730007A08C700D5004608D4003E08D3003D08EB
:10374000D2000330D6008A11831205218A15831610
:10375000D501E030D400D301D2010330D6008A1164
:10376000831205218A158316C301420843020318F8
:10377000D32B4108C10AC10AC400D501E030D400EE
:10378000D301D2010330D6008A11831205218A1594
:1037900083164408840077088000840A7808800033
:1037A0000230C307B52B8312D52B8A150A16FF2BBF
:1037B0000A148A140A118207762B8316B601831223
:1037C0002C088316B50083122B088316B4008312CD
:1037D0002A088316B30083122D08EF0083163608DB
:1037E000BA003508B9003408B8003308B7002D30E6
:1037F000BB0083126F088316BC008312652BC43094
:10380000A9000430EF070A128A1169200A168A15E6
:103810008A150A16B82EFF308316DE000A128312AC
:10382000C1270A16F8080319762C20302802FF3E1B
:103830000318762C013E792C83163B08C1003A0808
:10384000C0003908BF003808BE003C08C2003D086F
:10385000C3000310C00CBF0CBE0C3E08F7003F08AD
:10386000F80040081F39F90041080039FA003E0805
:10387000C5003F08C6007908D038C7007A08C800DC
:10388000D5004708D4003F08D3003E08D2000330DB
:10389000D6008A11831205218A158316C4014308B4
:1038A00044020318742C4208C20AC20A8400840A23
:1038B0000008FA0084030008C5007A08C600F0304A
:1038C000C700C8014808D5004708D4004608D300FF
:1038D0004508D2000330D6008A11831205218A15CB
:1038E00002308316C4074F2C8312762C8A150A16D1
:1038F0009F2C0A108A100A1582071C2C8316B60109
:1039000083122C088316B50083122B088316B4008B
:1039100083122A088316B300043083126F028316C1
:10392000B7003608BB003508BA003408B9003308C0
:10393000B8002D30BC003708BD0083120B2C0730B7
:10394000A9000130EF000A128A1169200A168A15AF
:103950008A150A16BE2E2A308316B20097308312BB
:10396000A90083163208B3008A11831293218A15A5
:10397000831633088400840A790880008403780859
:10398000800003308312EF000A128A1169200A16A0
:103990008A158A150A16C42EFF308316DE000A1215
:1039A0008312C1270A16F8080319432D2030280274
:1039B000FF3E0318432D013E462D83163508B900FE
:1039C0003708BA003808BB000F30C000FC30BF0019
:1039D0008A1183125B278A1578088316BC000F3082
:1039E000C200FC30C1003908C3008A118312A62727
:1039F0008A158316BD013B083D020318382D3A088D
:103A00003D07BE000F30C000FD30BF008A11831299
:103A10005B278A1583163E088400780880000130F1
:103A20003D073A07BF008A1183123C278A15831687
:103A30003F0884007808800002303D073A07BF0045
:103A40008A1183123C278A1583163F088400780860
:103A50008000B90A0F30C200FC30C1003908C30031
:103A60008A118312A6278A1503308316BD07FB2C03
:103A70000F30C200FC30C1003C08C3008A11831221
:103A8000A6278A15432D8A150A16662D0A148A1050
:103A90000A158207DD2C2A308316B20083122C0807
:103AA000EF00831632088400840A0008B4008403FF
:103AB0000008B3003408B6003308B5002C30B70056
:103AC00083126F088316B8008312CC2CE630A9004D
:103AD0000330EF070A128A1169200A168A158A151F
:103AE0000A16CA2EFF308316DE000A128312C1277F
:103AF0000A16F8080319E82D20302802FF3E0318A3
:103B0000E82D013EEB2D83163608BA003808BB00BD
:103B10003908BC000F30C000FC30BF008A1183128E
:103B20005B278A1578088316BD00BE013C083E025B
:103B30000318DD2D3A08BA0ABF000F30C200FC306E
:103B4000C1003F08C3008A118312A6278A15831675
:103B50003B083E0784000008BF000F30C200FD3064
:103B6000C1003F08C3008A118312A6278A150130BD
:103B700083163E073B0784000008C0000F30C200D8
:103B8000FE30C1004008C3008A118312A6278A159F
:103B9000023083163E073B0784000008C0000F3048
:103BA000C200FF30C1004008C3008A118312A6275B
:103BB0008A1503308316BE07962D0F30C200FC30E5
:103BC000C1003D08C3008A118312A6278A15E82D7B
:103BD0008A150A160A2E0A148A100A158207832DDE
:103BE0002A308316B20032088400840A0008B40028
:103BF00084030008B300033083126F028316B500FC
:103C00003408B7003308B6002C30B8003508B900C6
:103C10008312722D0730A9000130EF000A128A11B9
:103C200069200A168A158A150A16D02E8316B20143
:103C30003208033C031C682EB4013208B3000310A1
:103C4000320DF700B500350A0A128A1183123520A9
:103C50000A168A15FA00831635080A128A11831289
:103C600035200A168A158316B6007A08B70033087D
:103C7000831203178D00831603133408831203176E
:103C80008F00831603133608831203178C008316E4
:103C900003133708831203178E0083168C170C1535
:103CA000831203130B08F8008B1383160317553088
:103CB0008D00AA308D008C14000000008C185E2E40
:103CC0000C117808831203138B048316B20A182E82
:103CD0008A01831282018A150A16D62E8316B1082C
:103CE000031DDB2E83122908523C031D7B2E8A11F3
:103CF000872A8A15DA2E2908533C031D832E8A1140
:103D0000152B8A15DA2E2908543C031D8B2E8A1197
:103D1000F52B8A15DA2E2908553C031D932E8A119E
:103D2000C12C8A15DA2E2908563C031D9B2E8A11B8
:103D3000002F8A15DA2E2908603C031DA12E872941
:103D4000DA2E2908613C031DA72EF729DA2E29084F
:103D5000623C031DAD2E822ADA2E2908633C031D26
:103D6000B32E432BDA2E2908653C031DB92EDD2B1B
:103D7000DA2E2908643C031DBF2E7E2CDA2E29087A
:103D8000663C031DC52EAB2CDA2E2908673C031DAB
:103D9000CB2E4B2DDA2E2908683C031DD12EF02D99
:103DA000DA2E2908313C031DD72E162EDA2E8A1161
:103DB000E82F8A15831683128A150A164F2F84015D
:103DC0001F308305073083169F004030990026304E
:103DD0009800903083129800403083169900263066
:103DE0009800903083129800403083169900263056
:103DF0009800903083129800403083169900263046
:103E00009800903083129800403083169900263035
:103E100098009030831298007130F0000230F10069
:103E2000F4100714071499308316870010308600A9
:103E30000B308500B530831290008F018E01831600
:103E40000C14C03083128B040F30F700073081014F
:103E5000813084000008F0390738800064000008D1
:103E6000F039770480000A128A114B200A168A154D
:103E70000A128A11B2200A168A150B138B138B1B98
:103E80003E2F83160C108312061564008A11002839
:103E90008A1578088316B000B10083126E2E452F64
:103EA0006300FF3FFF3FFF3FFF3FFF3FFF3FFF3FFD
:103EB000FF3FFF3FFF3FFF3FFF3FFF3FFF3FFF3F12
:103EC000FF3FFF3FFF3FFF3FFF3FFF3FFF3FFF3F02
:103ED000FF3FFF3FFF3FFF3FFF3FFF3FFF3FFF3FF2
:103EE000FF3FFF3FFF3FFF3FFF3FFF3FFF3FFF3FE2
:103EF000FF3FFF3FFF3FFF3FFF3FFF3FFF3FFF3FD2
:103F0000FF3FFF3FFF3FFF3FFF3FFF3FFF3FFF3FC1
:103F1000FF3FFF3FFF3FFF3FFF3FFF3FFF3FFF3FB1
:103F2000FF3FFF3FFF3FFF3FFF3FFF3FFF3FFF3FA1
:103F3000FF3FFF3FFF3FFF3FFF3FFF3FFF3FFF3F91
:103F4000FF3FFF3FFF3FFF3FFF3FFF3FFF3FFF3F81
:103F5000FF3FFF3FFF3FFF3FFF3FFF3FFF3FFF3F71
:103F6000FF3FFF3FFF3FFF3FFF3FFF3FFF3FFF3F61
:103F7000FF3FFF3FFF3FFF3FFF3FFF3FFF3FFF3F51
:103F8000FF3FFF3FFF3FFF3FFF3FFF3FFF3FFF3F41
:103F9000FF3FFF3FFF3FFF3FFF3FFF3FFF3FFF3F31
:103FA000FF3FFF3FFF3FFF3FFF3FFF3FFF3FFF3F21
:103FB000FF3FFF3FFF3FFF3FFF3FFF3FFF3FFF3F11
:103FC000FF3FFF3FFF3FFF3FFF3FFF3FFF3FFF3F01
:103FD000FF3FFF3FFF3FFF3FFF3FFF3FFF3FFF3FF1
:103FE000FF3FFF3FFF3FFF3FFF3FFF3FFF3FFF3FE1
:103FF000FF3FFF3FFF3FFF3FFF3FFF3FFF3FFF3FD1
:08400000FF3FFF3FFF3FFF3FC0
:104200002000FF00FF00FF00FF00FF00FF00FF0095
:10421000FF00FF00FF00FF00FF00FF00FF00FF00A6
:10422000FF00FF00FF00FF00FF00FF00FF00FF0096
:10423000FF00FF00FF00FF00FF00FF00FF00FF0086
:10424000FF00FF00FF00FF00FF00FF00FF00FF0076
:10425000FF00FF00FF00FF00FF00FF00FF00FF0066
:10426000FF00FF00FF00FF00FF00FF00FF00FF0056
:10427000FF00FF00FF00FF00FF00FF00FF00FF0046
:10428000FF00FF00FF00FF00FF00FF00FF00FF0036
:10429000FF00FF00FF00FF00FF00FF00FF00FF0026
:1042A000FF00FF00FF00FF00FF00FF00FF00FF0016
:1042B000FF00FF00FF00FF00FF00FF00FF00FF0006
:1042C000FF00FF00FF00FF00FF00FF00FF00FF00F6
:1042D000FF00FF00FF00FF00FF00FF00FF00FF00E6
:1042E000FF00FF00FF00FF00FF00FF00FF00FF00D6
:1042F000FF00FF00FF00FF00FF00FF00FF00FF00C6
:10430000FF00FF00FF00FF00FF00FF00FF00FF00B5
:10431000FF00FF00FF00FF00FF00FF00FF00FF00A5
:10432000FF00FF00FF00FF00FF00FF00FF00FF0095
:10433000FF00FF00FF00FF00FF00FF00FF00FF0085
:10434000FF00FF00FF00FF00FF00FF00FF00FF0075
:10435000FF00FF00FF00FF00FF00FF00FF00FF0065
:10436000FF00FF00FF00FF00FF00FF00FF00FF0055
:10437000FF00FF00FF00FF00FF00FF00FF00FF0045
:10438000FF00FF00FF00FF00FF00FF00FF00FF0035
:10439000FF00FF00FF00FF00FF00FF00FF00FF0025
:1043A000FF00FF00FF00FF00FF00FF00FF00FF0015
:1043B000FF00FF00FF00FF00FF00FF00FF00FF0005
:1043C000FF00FF00FF00FF00FF00FF00FF00FF00F5
:1043D000FF00FF00FF00FF00FF00FF00FF00FF00E5
:1043E000FF00FF00FF00FF00FF00FF00FF00FF00D5
:1043F000FF00FF00FF00FF00FF00FF00FF00FF00C5
:00000001FF
